:100000000C9406030C944D030C944D030C944D0377
:100010000C944D030C944D030C944D030C944D0320
:100020000C944D030C944D030C944E210C940A2116
:100030000C944B220C944D030C944D030C944D03E3
:100040000C944D030C944D030C944D030C944D03F0
:100050000C944D030C9427220C944D030C944D03E7
:100060000C944D030C944D030C944D030C944D03D0
:100070000C944D030C944D030C944D030C944D03C0
:100080000C944D030C944D030C944D030C944D03B0
:100090000C944D030C944D030C944D030C944D03A0
:1000A0000C944D030C944D030C944D03050109026F
:1000B000A10185020901A1000509190129081500FE
:1000C0002501950875018102050109300931158165
:1000D000257F95027508810609381581257F9501D0
:1000E00075088106050C0A38021581257F95017572
:1000F000088106C0C005010980A101850319012AF4
:10010000B700150126B700950175108100C0050CD8
:100110000901A101850419012AA002150126A002E6
:10012000950175108100C005010906A1018506052C
:100130000719E029E71500250195087501810205D9
:1001400007190029EF1500250195F07501810205B9
:10015000081901290595057501910295017503910D
:1001600001C00660FF0961A1010962150026FF00B8
:100170009520750881020963150026FF00952075FA
:10018000089102C005010906A101050719E029E748
:1001900015002501950875018102950175088101F9
:1001A0000507190029FF150026FF0095067508812F
:1001B000000508190129059505750191029501753C
:1001C000039101C0000000000000000000000000DA
:1001D000000000000000000000000000000000001F
:1001E00000000000000000007E0F00D4FFFFFFC7EA
:1001F0000000007800000000000000002A2B28000A
:1002000000000000000000000000000000000029C5
:10021000000000002C1E3420212224342627252E05
:10022000362D3738271E1F2021222324252633333D
:10023000362E37381F0405060708090A0B0C0D0E69
:100240000F101112131415161718191A1B1C1D2F35
:100250003130232D350405060708090A0B0C0D0E55
:100260000F101112131415161718191A1B1C1D2F15
:100270003130354C00047F3F1F64321464321478EF
:100280003C1E1E140A0500010101010101010101CA
:100290000202020202020202020303030303030337
:1002A0000304040404040404050505050506060604
:1002B0000606070707070708080808090909090AC1
:1002C0000A0A0B0B0B0C0C0C0D0D0D0E0E0E0F0F66
:1002D0000F101011111112121313141415151616F4
:1002E0001717181819191A1A1B1B1C1D1D1E1E1F63
:1002F0002020212222232424252626272829292AB2
:100300002B2C2D2D2E2F30313232333435363738D9
:10031000393A3B3C3D3E3F404142434445464748D5
:10032000494A4C4D4E4F50515354555658595A5BAB
:100330005D5E5F616264656668696B6C6D6F70724B
:10034000737577787A7B7D7E8082838587888A8CB7
:100350008E8F91939596989A9C9EA0A2A3A5A7A9EB
:10036000ABADAFB1B3B5B7BABCBEC0C2C4C6C9CBE2
:10037000CDCFD1D4D6D8DBDDDFE2E4E7E9EBEEF098
:10038000F3F5F8FAFDFFFFAA7F5540222325262822
:10039000292A2C2D2F3032333536383A3B3D3E401A
:1003A00042434547494A4C4E5051535557595A5C60
:1003B0005E6062646668696B6D6F71737577797B77
:1003C0007D7F81838587898A8C8E90929496989A76
:1003D0009C9E9FA1A3A5A7A8AAACAEAFB1B3B4B68B
:1003E000B8B9BBBCBEBFC1C2C3C5C6C7C9CACBCCE6
:1003F000CDCED0D1D2D2D3D4D5D6D7D7D8D9D9DAB9
:10040000DADBDBDBDCDCDCDCDCDDDDDDDDDCDCDC2D
:10041000DCDCDBDBDBDADAD9D9D8D7D7D6D5D4D355
:10042000D2D2D1D0CECDCCCBCAC9C7C6C5C3C2C12A
:10043000BFBEBCBBB9B8B6B4B3B1AFAEACAAA8A787
:10044000A5A3A19F9E9C9A98969492908E8C8A893F
:10045000878583817F7D7B79777573716F6D6B691C
:1004600068666462605E5C5A5957555351504E4CF1
:100470004A4947454342403E3D3B3A3836353332A0
:10048000302F2D2C2A292826252322350029002B20
:100490000001512A0036005300540055005600E375
:1004A000005F00600061005700E2005C005D005EDC
:1004B000000000E10059005A005B000000E000620B
:1004C00000630058000000005C0100010001000111
:1004D000000100010001000100010001004A00527A
:1004E000004B0001000100500000004F000000011F
:1004F000004D0051004E000000010049004C000179
:1005000000000001000100010001000100010001E4
:1005100000010001000100010001000100010001D3
:1005200000010001000100010000000100010001C4
:1005300000010000000100010001000100000001B5
:1005400000010001000100010001000100010001A3
:100550000001000100010001000100010001000193
:100560000001000100000001000100010001000085
:10057000000100010001000100000009025B00030E
:100580000100A0FA09040000010301010009211182
:100590000100012240000705810308000A09040147
:1005A00000020300000009211101000122220007BE
:1005B000058203200001070503032000010904024E
:1005C00000010300000009211101000122B600070B
:1005D00005840320000A120100020000000864697B
:1005E00060600100010200010E034D006F006E000B
:1005F00074006500780000000E03490064006F007D
:10060000620061006F0000000403090411241FBE92
:10061000CFEFDAE0DEBFCDBF04B603FE27C0809186
:10062000CF029091D002A091D102B091D202873036
:10063000904BA740B04BD1F41092CF021092D00251
:100640001092D1021092D20214BE84B7877F84BF69
:100650000FB6F894A895809160008861809360003F
:10066000109260000FBEE0E0F8E3099511E0A0E011
:10067000B1E0E6E3F2E502C005900D92AC38B107B7
:10068000D9F722E0ACE8B1E001C01D92AF3CB2075F
:10069000E1F70E9472220C94E2280C940000E8ED2D
:1006A000F0E080818E7F80831092E2001092DA0069
:1006B0001092E100A0EEB0E08C9181608C9380817B
:1006C0008F77808319BCA7EDB0E08C918E7F8C93DF
:1006D00080818F7E808310929C0208952091E40097
:1006E0003091E50095E6A9012091EC00822F817000
:1006F00020FF06C08091E80080FF06C080E00895DA
:100700002091E80022FD1AC08091C102882389F05F
:10071000853089F08091EB0085FD0FC02091E400C9
:100720003091E50042175307F9F29150E1F684E069
:10073000089582E0089583E0089581E00895EF929E
:10074000FF920F931F93CF937C018B010E946E0346
:10075000C82F811117C08091E80085FD0BC08091E2
:10076000E8008E778093E8000E946E03882399F357
:10077000C82F08C0F70181917F018093F1000150DB
:10078000110949F78C2FCF911F910F91FF90EF9096
:1007900008958091C30287FF13C08091E80082FF13
:1007A00006C08091E8008B778093E80004C08091B8
:1007B000C1028111F2CF08958091C1028823D9F33B
:1007C0008091E80080FFF8CF8091E8008E77ECCF31
:1007D000982F9093E900242F762F50E0891731F05D
:1007E0007091EC002091ED005091F00021FD07C0C8
:1007F0009F5F973071F78093E90081E00895309111
:10080000EB003E7F3093EB003091ED003D7F309365
:10081000ED003091EB0031603093EB007093EC0011
:100820002093ED005093F0002091EE0027FDE0CFE3
:1008300080E00895CF92DF92EF92FF920F931F9383
:10084000CF93DF93C8EDD0E088818F7E8883E7ED7A
:10085000F0E080818160808384E082BF81E08093CA
:100860009C0288818E7F888302EE10E0F80110825E
:100870001092DA0081EEC82ED12CF6011082888108
:100880008F77888388818068888388818F7D88833B
:1008900019BC1092C1021092C2021092C0021092B2
:1008A000BF0290EEE92EF12CF70180818B7F8083CF
:1008B00088818160888342E060E080E00E94E803F4
:1008C000F60180818E7F8083F80180818160808342
:1008D000808188608083F70180818E7F808388811A
:1008E00080618883DF91CF911F910F91FF90EF90EE
:1008F000DF90CF900895FC018091C9029091CA02C7
:1009000086179707A0F06115710529F49091E8000A
:100910009E779093E80090E06115710551F4911174
:1009200008C08091E80082FF34C080E00895BC01D7
:10093000F2CF8091C1028823C1F18530C1F180914D
:10094000E80083FD30C08091E80082FDEACF80910D
:10095000E80080FFE1CF8091F3002091F200382F72
:100960006115710519F02830310558F091E02830F3
:10097000310509F090E02091E8002E772093E800FF
:10098000CBCF81918093F100615071092F5F3F4F70
:10099000E7CF8091C102882341F0853041F08091FA
:1009A000E80083FFBECF81E0089582E0089583E0F0
:1009B0000895089580919E0208959C014FB7F89480
:1009C0008091930290919402A0919502B091960229
:1009D0004FBF821B930B08952FB7F8948091930219
:1009E00090919402A0919502B09196022FBF089524
:1009F00020919002309191022817390771F090935D
:100A0000910280939002E0918E02F0918F023097D4
:100A100021F00084F185E02D0994089520918C0245
:100A200030918D022817390771F090938D028093D1
:100A30008C02E0918E02F0918F02309721F00680B7
:100A4000F781E02D09940895E0918E02F0918F02D4
:100A5000309721F00190F081E02D099480E0089515
:100A60008F929F92AF92BF92EF92FF920F931F933C
:100A7000CF93DF938430B8F5811136C09091800018
:100A80009F7D909380002E98A0918600B091870062
:100A9000282F30E00E944B2823E030E040E050E077
:100AA0000E94142889019A01809186009091870004
:100AB0006CE070E00E94EC2760177107D8F0C80165
:100AC00069E070E00E94EC2770938B0060938A00CD
:100AD000DF91CF911F910F91FF90EF90BF90AF905A
:100AE0009F908F90089583E0909180009062909302
:100AF0008000CACF8091860090918700E0908600A8
:100B0000F0908700E0918600F0918700C6E0D0E089
:100B1000BE010E94EC27060F171F211D311D480141
:100B2000590185E0880C991CAA1CBB1C8A95D1F739
:100B3000C701BE010E94EC279F0150E040E0260F54
:100B4000371F411D511DC501B4010E9414284901E0
:100B50005A01E0918600F0918700CA01B9010E9414
:100B6000CE279B01AC01DF010E9461289B01AC01F3
:100B7000C501B4010E94CE272FE096958795779501
:100B800067952A95D1F7009186001091870030E093
:100B900020E0061717072807390708F095CF60915E
:100BA00086007091870090CF282F220F220F220FEE
:100BB00090918B029770922B90938B02987F21E0FB
:100BC00009F420E090918B0220FB90F990938B0226
:100BD0000C943005FA01811101C0FB0109940895BC
:100BE00080918602982F9E7F29F481708260809385
:100BF000860208958A34E8F381708864F8CFAF9252
:100C0000BF92DF92EF92FF920F931F93CF93DF93E8
:100C1000082F162FE901E42FF0E0EA57FD4F61118C
:100C200010C0E4915E2F4E2F4983E8835A83DF91F1
:100C3000CF911F910F91FF90EF90DF90BF90AF90F9
:100C40000895E62EF12C4491D42EE42FF0E026E016
:100C5000829FC00111242FEF30E0B9010E94EC27E0
:100C6000802F90E0880F991F55E5569FD001579F20
:100C7000B00D11248A1B9B0B982F990F890F5901D6
:100C8000AE18BF08AE9ED001AF9EB00DBE9EB00D97
:100C900011245B2F189F80011124012F1127590166
:100CA000A01AB10AAE9E8001AF9E100DBE9E100D1F
:100CB00011245901A81AB108AE9CC001AF9C900D37
:100CC000BE9C900D1124892F9927281B390B2E9F2C
:100CD000C0012F9F900D3E9F900D1124E92F62308F
:100CE0007105A1F050F46115710509F49DCF6130D3
:100CF000710581F0EB2F512F97CF6430710569F0AA
:100D000080F06630710509F48FCFF4CFE42F4B2FBC
:100D1000592F8ACFE42F412F87CFEB2F542F492F04
:100D200083CF4B2F5D2DE12F7FCF0E94EC049C01E0
:100D300090911A0280911B02982B21F03093170298
:100D40002093160290911C0280911D02982B21F095
:100D50003093150220931402E0918E02F0918F02DD
:100D6000309749F082E0809318020480F581E02DED
:100D700088E192E00994089540911A02803F59F465
:100D800080911B0287FF0DC010921B0241110BC006
:100D90001092120208C0813F81F480911B02181644
:100DA0009CF3442381F080911C0290911D02892BB9
:100DB00009F05AC0109211020895823F49F447FF8A
:100DC000F0CF10921A0280911B028111ECCFE0CF7C
:100DD000833F19F41416ACF3E4CF90911C02893FC1
:100DE00029F41916F4F610921C02DBCF8A3F19F48D
:100DF00097FFD7CFF8CF90911D028B3F29F497FF33
:100E0000D0CF10921D02CDCF8C3F19F41916CCF320
:100E1000C8CF9CE0980F953090F4845F990B21E047
:100E200030E0B90102C0660F771F8A95E2F7CB0167
:100E3000809590911902892380931902B2CF8D3F3A
:100E400031F4809113028E7F80931302AACF8E3FDC
:100E500021F4809113028D7FF7CF8F3F09F0A1CF4E
:100E6000809113028B7FF0CF08958091130280FD53
:100E700016C081FD16C082FD16C080911102882324
:100E8000A1F0883280F428E0829FC001112468E23A
:100E900070E00E940028862F672B39F0089582E0C9
:100EA000089584E0089588E0089581E00895809190
:100EB000130280FD14C081FD14C082FD16C0809114
:100EC0001202882381F0843180F422E3829FC001E2
:100ED000112464E170E00E940028862F08958CE0C0
:100EE000089589E1089585E0089582E30895803F9B
:100EF00031F40E945707819580931B020895813F2A
:100F000019F40E945707F8CF823F31F40E94570727
:100F1000819580931A020895833F19F40E94570720
:100F2000F8CF893F29F40E94350780931C02089569
:100F30008A3F21F40E9435078195F7CF8B3F31F42A
:100F40000E943507819580931D0208958C3F19F406
:100F50000E943507F8CF9CE0980F953070F4845FBD
:100F6000990B21E030E001C0220F8A95EAF78091C9
:100F70001902822B8093190208958D3F31F48091DC
:100F8000130281608093130208958E3F21F48091B3
:100F900013028260F7CF8F3FB9F78091130284600C
:100FA000F1CF80E00895F894E82FE295EF70F0E03B
:100FB00031A1282F2F7081E090E001C0880F2A9581
:100FC000EAF7982F9095932391A392A1892B82A35E
:100FD000789408959091970292FF06C0282F287167
:100FE0002830F9F4877F846093FF06C0282F28718A
:100FF0002831F1F4877E84612091980220FF06C099
:10100000382F38713830D9F4877F816021FF06C0CE
:10101000282F28712831D1F4877E816194FD877E45
:101020000895282F24712430F9F68B7F8860DCCF57
:10103000282F2471243101F78B7E8861DDCF382F72
:101040003171313019F78E7F8860E0CF282F217100
:10105000213121F78E7E8861E1CFCF93DF93EC01C0
:1010600082389105A9F1D8F58133910509F496C02C
:1010700048F58932910509F48AC08A9709F495C028
:10108000C11521E5D20708F0BCC0C11530E5D30772
:1010900008F014C1C83ED10508F09CC0C03ED1057F
:1010A00060F5C83AD10508F087C0C53AD10508F007
:1010B000FDC0C130D10509F12097F9F0C430D10548
:1010C000E0F440C08533910509F45AC0C997C1F6D0
:1010D00080919702837089F0C0EED0E00EC0833E0D
:1010E000910599F170F4803E910501F1823E9105E0
:1010F00039F68091970282FD21C0CE01DF91CF9118
:101100000895863E910561F1873E910571F1843E17
:10111000910509F0B5CF8091980281FFEECF8091C3
:101120009702C7EED0E084FD0DC0E7CF8091970213
:1011300080FD12C19091980290FFDFCFC3EED0E006
:1011400084FFDBCFD0E0C0E0D8CF8091970282FD52
:1011500006C19091980290FDBFCF84FFCECFF2CF11
:101160008091970283FDDDCFC8CF8091970283FDE8
:10117000F9C09091980291FFF0CFC4EED0E0BDCFBE
:101180008091970285FFB9CFC9E2D0E0B6CF8091B8
:10119000970285FFB2CFC5E3D0E0AFCF8091970231
:1011A00086FFABCFCAE2D0E0A8CF8091970286FF3E
:1011B000A4CFC1E3D0E0A1CFCF3BD10518F6C85AE8
:1011C000D0E0CC0FDD1FC25EDE4F0990D881C02D6C
:1011D000D46493CFC11540E2D40758F4C11581E01F
:1011E000D80708F08ACFC03FD10508F4ABCFD0654F
:1011F00084CFC11590E4D90708F4A4CFDF70D06A7A
:101200007CCFC11525E5D20700F5C11534E5D3071C
:1012100008F08AC0C11543E5D40708F071C0C115B4
:1012200082E5D80708F467C0CE018370992721E0D2
:1012300030E002C0220F331F8A95E2F7C695C695AB
:1012400080E2C89FE001112452C0C11599E5D90779
:10125000A8F4C11528E5D20708F06BC0C11536E522
:10126000D30708F06FCF8C2F0E94EA07C82FD0E079
:10127000DC2FCC27CC27DF71D0623FCFC1154AE5E8
:10128000D40708F45BC0CE0190568115904208F057
:1012900059CF8D2F8F710E94EA0790E0982F8827F1
:1012A00088279F719C012C2BE901E6CFC55AD0E01D
:1012B000C55EDE4FC881D0E0D0641FCFCE01E4E030
:1012C00096958795EA95E1F783702C2F26952695BC
:1012D000237040E2249F90011124382B8C2F8370BF
:1012E000C1E0D0E002C0CC0FDD1F8A95E2F7C22B2F
:1012F000D32BDC6802CFDC2FCC27C16FD06AFDCEA8
:10130000CE018370992721E030E002C0220F331F05
:101310008A95E2F7C695C69590E2C99FE00111242F
:10132000C22BD32BDA68E9CEDC2FCC27C46FD06A6E
:10133000E4CEDC2FCC27C06FD06ADFCE8C2F8F702D
:101340000E94EA0734E0D695C7953A95E1F7CF7049
:101350009C2FEC01D069D1CEC9E3D0E0CECEC2EE55
:10136000D0E0CBCEC6EED0E0C8CE8091F70181119F
:101370001092F701089580959091F601982390932B
:10138000F60108958091F6019091F501892B9091D5
:10139000F401892B80938E019091F7019923A1F09C
:1013A000892B80938E0180911A01882341F18091CD
:1013B000970287FF24C08EE1E0E9F1E090E08150E0
:1013C00000F591110E94B509E0918E02F0918F0213
:1013D0003097E1F080911A01882359F080919702AB
:1013E00087FF07C080918E0180938F0186E08093F4
:1013F0008E010280F381E02D8EE891E0099486E071
:10140000DBCF21912223D9F29F5FD9CF089590910C
:101410001A019923D1F09091970297FF16C0E82FF7
:10142000E695E695E695EE31E0F4F0E0E257FE4F02
:10143000282F277081E090E001C0880F2A95EAF7F5
:1014400080959281892382830895E0E9F1E091916A
:10145000891303C0DF0111971C9291E0E639F90767
:10146000B1F7089590911A019923C1F090919702D4
:1014700097FF14C0E82FE695E695E695EE31F8F46F
:10148000F0E0E257FE4F877021E030E001C0220F0C
:101490008A95EAF78281822B82830895A0E9B1E0E0
:1014A000EFEF90E02D91821751F0EF3F19F42111E9
:1014B00001C0E92F9F5F9630A9F7EF3F09F4089527
:1014C0000E2E000CFF0BE257FE4FE6CF8091F2018B
:1014D0009091C101981301C008958F5F8770FACF72
:1014E000E92FEE0FEE0F9E0F890F982F97708695BC
:1014F0008695869523E0829FF0011124E155FE4FE9
:1015000050E040E080E0219130E0092E02C03695A5
:1015100027950A94E2F721703327042E01C0220F89
:101520000A94EAF7822B4F5F5F4F4330510559F71A
:101530000895E92FEE0FEE0F9E0F890F982F9770E9
:1015400041E001C0440F9A95EAF786958695869505
:1015500093E0899FF0011124E155FE4F30E020E037
:1015600070E05191DF011197CB01022E02C09695D8
:1015700087950A94E2F781708195852784238527D2
:101580008C932F5F3F4F2330310559F7089590E03A
:1015900080E00E940E0590E080E00E94F804109226
:1015A000F5011092F4010E94C20986E0E8E1F2E040
:1015B000DF011D928A95E9F7109212021092110232
:1015C000109213020C9495068093CE020C94C70AD5
:1015D0008091CE02982F9670963019F488600C9402
:1015E000E40A877FFCCF21E030E001C0220F8A951A
:1015F000EAF720958091CE0282230C94E40A909120
:10160000F301809589238093F301282F277091F4AB
:10161000282F082E000C330B9217130659F09091C7
:10162000980292FD07C08595859585950E94F30ADD
:101630001092F301089521E030E001C0220F8A9555
:10164000EAF78091CE02822B0C94E40A8093F80191
:101650000C94C70A882321F00E94BB090C94C2098C
:101660000895882339F09091F601982B9093F60114
:101670000C94C2090895882309F452C0823871F489
:101680000E94240581FF4CC089E30E94320A0E9417
:10169000C20989E30E94070A0C94C209833859F4ED
:1016A0000E94240580FF3CC083E50E94320A0E940C
:1016B000C20983E5EFCF843859F40E94240582FFE4
:1016C0002FC087E40E94320A0E94C20987E4E2CF59
:1016D0009CEF980F913AF0F290E2980F983050F406
:1016E000877091E001C0990F8A95EAF7892F0E94CF
:1016F000BB09D2CF9BE5980F933020F490E080E0B7
:101700000C940E0598E5980F973120F490E080E056
:101710000C94F804803F20F00E94BC060C949506BF
:1017200008958093990270939B0260939A0280912E
:10173000C1028430F9F48093E9008FEF9091E800C2
:10174000815095FD06C095ED9A95F1F70000811145
:10175000F5CF8091E80085FF0DC050E040E063E0E8
:1017600070E089E992E00E949F038091E8008E7703
:101770008093E8000895BC0184E00C94910BBC01B7
:1017800083E00C94910B9C0184E08093E9009FEF2F
:101790008091E800915085FD06C085ED8A95F1F7AE
:1017A00000009111F5CF8091E80085FF0CC050E05A
:1017B00040E066E070E0C9010E949F038091E8006C
:1017C0008E778093E8000895CF93DF93EC018091AA
:1017D0001A018823B1F18091970287FF32C060E23D
:1017E00084E08093E9008FEF9091E800815095FDAF
:1017F00006C095ED9A95F1F700008111F5CF809123
:10180000E80085FF1BC080911A0170E050E040E0C5
:10181000811104C050E040E068E070E0CE010E9419
:101820009F038091E8008E778093E80080E2FE01BC
:10183000AFE9B2E001900D928A95E1F7DF91CF9187
:10184000089568E081E0CDCF81E08093E00080E200
:101850008093D8001092C9008FE19EE40197F1F7C0
:1018600000C0000087E090EBDC018093CF029093F2
:10187000D002A093D102B093D20288E19CE00FB6CF
:10188000F894A895809360000FBE90936000FFCFFE
:101890008091860280FD0AC0E9E2F2E011821082A6
:1018A0001282339652E0E638F507C1F7219A35B136
:1018B0003D7F25B122604FB7F89489E292E0FC01A8
:1018C0005191CF0168E025B9000000C057FF35B93C
:1018D000550F000000C000C000C035B900C06A95B7
:1018E00091F7F2E086389F0751F74FBF8FE594E0FC
:1018F0000197F1F700C000000895EF92FF920F9357
:101900001F93CF93DF938C01C9E2D2E0F12CE12C3D
:10191000F80194816091880280918702FFE0EF16C0
:10192000F104FCF49923F9F09E01409189020E9490
:10193000FF052FEFE21AF20A23968FE1E816F10471
:1019400039F70E94480CF801848190E0019681707B
:1019500099278483DF91CF911F910F91FF90EF9092
:101960000895992309F39E0140E0E1CF8F929F9261
:10197000AF92BF92CF92DF92EF92FF920F931F939D
:10198000CF93DF93EC014C81042F10E09801D80134
:101990000E944B289B01AC010E9461284B015C0115
:1019A000E0E2F0E0E01BF10BA5E5B0E0AC019B014B
:1019B0000E9461286B017C019F01DF010E94432886
:1019C0009B01AC010E946C289B01AC01280D391DC4
:1019D0004A1D5B1DC701B6010E941428F22E822FFA
:1019E00090E039E23F15D8F143E0249F90011124A3
:1019F00035952795122F109599E2C92E92E0D92E90
:101A000000E085E5E82EEF188E2D01FD8F2D960163
:101A1000412F609188020E94FF050F5F53E0C50EC1
:101A2000D11C0F3189F70E94480C9C8181E09923D9
:101A300019F0903219F48FEF8093190180911901F8
:101A4000890F8C83DF91CF911F910F91FF90EF90C1
:101A5000DF90CF90BF90AF909F908F90089525E535
:101A600030E0A901481B590BCA019A01220F331F0C
:101A7000280F391F37FFBCCF2F5F3F4FB9CF0F93D0
:101A80001F93CF93DF93C9E2D2E0FE01118210824F
:101A90001282339682E0E638F807C1F710E000E0E2
:101AA00080912702082E000C990B081719078CF15A
:101AB00080911801082E000C990B801791074CF1AA
:101AC0009E014091890260918802809187020E9464
:101AD000FF050F5F1F4F23960F31110509F70E9475
:101AE000480C8091170190912702980F909327023C
:101AF00020911801280F20931801121614F49E311A
:101B00001CF0819580931701DF91CF911F910F9168
:101B10000895198218821A82DCCFBF92CF92DF9289
:101B2000EF92FF920F931F93CF93DF93FC0182817B
:101B3000DD24DA9480FD02C0DD24D39409E212E0B2
:101B4000D0E0C0E02FE1B22EF801118210821282A3
:101B500094E0E92EF12CC12C809126028C0D80326C
:101B60000CF43DC06B2D0E94DE27892F082E000C3F
:101B7000990B8C179D0791F4809189028E9DA0018D
:101B80008F9D500D11245595479555954795980172
:101B900060918802809187020E94FF05CD0CF1E0E0
:101BA000EF1AF108C9F621960D5F1F4FCF31D1050D
:101BB00059F60E94480C8091260291E0D91215C076
:101BC000811111C08EE180932602DF91CF911F9188
:101BD0000F91FF90EF90DF90CF90BF90089587FF17
:101BE000C5CF815EC3CF8150EECF90E00196BE019C
:101BF0000E940028E8CFEF92FF921F93CF93DF93CC
:101C0000EC0189E2E82E82E0F82E10E08C81970149
:101C10004091890260918802810F0E94FF05185F40
:101C200083E0E80EF11C183F89F70E94480C9A8166
:101C30008C8190FF08C08F5F8C83DF91CF911F91C3
:101C4000FF90EF9008958150F7CF9091860290FF1A
:101C50000CC0E9E2F2E0818360834283339692E034
:101C6000E638F907C1F70C94480C08950F931F93B9
:101C7000CF93DF9300D00F92CDB7DEB78C01809168
:101C8000280281110AC09E012F5F3F4F4FEF6FEF77
:101C90000E94FF058A8180932802F80164816130E7
:101CA00069F08091280240E0662361F040E06230F4
:101CB00011F44091280280E060E004C060912802A5
:101CC00040E080E00E94250EF801848190E00196BA
:101CD00063E070E00E94002884830F900F900F90C3
:101CE000DF91CF911F910F910895CF93DF9300D093
:101CF0000F92CDB7DEB79091860290FF0AC09E0189
:101D00002F5F3F4F0E94FF054B8169818A810E94AE
:101D1000250E0F900F900F90DF91CF910895CF93E4
:101D2000DF93EC01E6E8F2E0438162818C810E945E
:101D3000750E8C818F5F8C83DF91CF910895CF9347
:101D4000DF93EC01EC81F0E0E557FC4F4491E6E8CD
:101D5000F2E0628181810E94750E8C818F5F8C839D
:101D6000DF91CF910895CF93C82F882309F4AEC097
:101D70008238C1F40E94240581FDA8C089E30E9435
:101D8000320A0E94C2092FEF81EE94E02150804078
:101D90009040E1F700C0000089E30E94070ACF915C
:101DA0000C94C2098338A1F40E94240580FD8EC0E2
:101DB00083E50E94320A0E94C2092FEF81EE94E06F
:101DC000215080409040E1F700C0000083E5E5CF5E
:101DD0008438A1F40E94240582FD78C087E40E9423
:101DE000320A0E94C2092FEF81EE94E02150804018
:101DF0009040E1F700C0000087E4CFCF8CEF8C0F5C
:101E0000813A88F580911A01882301F18091970227
:101E100087FF1CC0EC2FE695E695E695F0E0E257CB
:101E2000FE4F828190E04C2F477021E030E002C0ED
:101E3000220F331F4A95E2F782239323892B79F0EF
:101E40008C2F0E94070A0E94C20909C0E0E9F1E054
:101E50008191C817A9F321E0E639F207C9F78C2F61
:101E60000E94320A9CCF80E28C0F883068F4C770E1
:101E700021E030E001C0220FCA95EAF78091F60117
:101E8000822B8093F6018BCFEBE5EC0FE33040F42F
:101E9000F0E0E55EFE4F808190E0CF910C940E055E
:101EA000E8E5EC0FE73150F4F0E0EE0FFF1FE25EE3
:101EB000FE4F80819181CF910C94F804C03F30F0A7
:101EC0008C2F0E947707CF910C949506CF9108959F
:101ED0001F93CF93DF93182FD0E0C0E0893311F424
:101EE000C0E5D0E0812F0E94B30E209731F4812FFE
:101EF000DF91CF911F910C943B0B8FE99FE00197ED
:101F0000F1F700C000002197F0CF0F931F93CF93FC
:101F1000DF93C62FD42F022FFC0182818823A1F0EA
:101F20006093CD020E94EC049093CC028093CB028C
:101F3000C77081E001C0880FCA95EAF7DF91CF91A1
:101F40001F910F910C94310B8091CD02681335C015
:101F50008091CB029091CC020E94DD04883C9105D7
:101F600060F510E21D0FCD17B9F080E28C0F8830BC
:101F700040F4C77081E001C0880FCA95EAF70E945B
:101F80002A0B183048F481E09D2F977001C0880F0C
:101F90009A95EAF70E94310B802F0E94680F183043
:101FA00098F4D77081E001C0880FDA95EAF7DF91E5
:101FB000CF911F910F910C942A0BC77081E001C043
:101FC000880FCA95EAF7F3CFDF91CF911F910F9158
:101FD0000895CF93DF93C7E1D1E060E0CE010E9486
:101FE00094282196C11584E0D807B9F7DF91CF91E5
:101FF00008956F927F928F929F92AF92BF92CF92ED
:10200000DF92EF92FF920F931F93CF93DF938BE8B2
:10201000C82E84E0D82E9DE6E92EF12CE701EC973E
:1020200036011BC0F50185909490692DC8010E946E
:102030009428682DC80101960E94942882E0A80E79
:10204000B11C0E5F1F4FC017D10761F78AE0680E01
:10205000711C2A96CE15DF0529F08E010A50110950
:102060005301E0CF7E018CE3E80EF11C8CE3C80E37
:10207000D11C8DE5E81681E0F80681F6DF91CF915D
:102080001F910F91FF90EF90DF90CF90BF90AF9096
:102090009F908F907F906F900895CF93C82F6FEF90
:1020A000811162E283E290E00E9494286FEFC111F7
:1020B00062E084E290E00E9494286FEFC11164E135
:1020C00085E290E0CF910C94942880E00E944D101E
:1020D00060E086E290E00E9494280E94F90F0E943E
:1020E000E90F81E00C944D10682F86E090E00C948D
:1020F0009428CF93C0919802C2FB992790F9981722
:1021000099F080FBC2F9C09398026091970284E035
:1021100090E00E9494286C2F82E290E00E94942824
:1021200082E0CF910C94FF0ACF9108950F931F93F3
:10213000CF93DF93C42FD0E0CC0FDD1F2AE0629F46
:10214000C00DD11D11243CE3839FC00DD11D11246E
:10215000CE0187960E948028082F10E0102F0027BC
:10216000CE0188960E9480289801282BC901DF9112
:10217000CF911F910F910895462F843038F4763017
:1021800028F4653018F4672F0C94961090E080E0E6
:102190000895CF92DF92FF920F931F93CF93DF9317
:1021A0006C010091CE028091F801082BC7E0D0E0CD
:1021B00010E0FC2EC8010C2E02C0959587950A945C
:1021C000E2F780FD0CC02197A0F7F12C8F2DDF9155
:1021D000CF911F910F91FF90DF90CF900895B6019E
:1021E0008C2F0E94BC100E942D08019761F3EECF46
:1021F000CF93DF93EC010E94C910BE010E94BC1076
:10220000DF91CF910C942D08FC01808191810E9477
:10221000F810292F2F7092959F7092509E3078F46D
:10222000E92FF0E0EC51F74D0C943628803F19F07F
:1022300020F4883E20F481E00895843FE1F380E0BB
:102240000895883EC0F3813FD1F7F5CF822F869560
:1022500086958695089583E290E00E9480288232D8
:1022600089F484E290E00E948028823059F485E26B
:1022700090E00E94802891E0843109F090E0892F5D
:102280008170089580E0FCCFCF9384E090E00E94BD
:102290008028C82F82E290E00E948028982F8C2FFF
:1022A000CF910895CF92DF92EF92FF926B017C0164
:1022B0000E94F005B701A60188E090E0FF90EF9042
:1022C000DF90CF900C94A6285F926F927F928F92AE
:1022D0009F92AF92BF92CF92DF92EF92FF920F93B5
:1022E0001F93CF93DF9300D00F92CDB7DEB7182F97
:1022F000762E042F622E9091860290FF29C0E92F3E
:10230000E695AE2FB0E0A95ABE4F8C91809324027F
:102310009E7F923081F59E012F5F3F4F812F0E945B
:10232000FF054B8169818A810E94250E10938702E7
:102330007092880200938902662051F060918602B3
:102340007091870280918802909189020E945211B7
:102350000F900F900F90DF91CF911F910F91FF90F1
:10236000EF90DF90CF90BF90AF909F908F907F9035
:102370006F905F900895823019F400918902D6CF52
:10238000863019F410918702D1CF8930D9F3893181
:1023900069F6E9518E2F8170582EE695F0E0EA57E4
:1023A000FC4FA590B490BB2489E2E82E82E0F82E81
:1023B000D12CC12C9FE1892E912CC601B4010E9421
:1023C000EC27812F511013C0860F9701402F672DE6
:1023D0000E94FF05CA0CDB1C83E0E80EF11C86E8B6
:1023E000E81682E0F80649F70E94480C9FCF861B4A
:1023F000ECCFE6E8F2E0438128E0421B08F440E03D
:1024000021E0628181810C946411E6E8F2E043816D
:1024100028E0420F08F44FEF21E0628181810C94A3
:102420006411E6E8F2E0628128E0621B08F460E0F3
:1024300021E0438181810C946411E6E8F2E062813D
:1024400028E0620F08F46FEF21E0438181810C9452
:102450006411E6E8F2E0818121E0438162818850E5
:102460000C946411E6E8F2E0818121E0438162810D
:10247000885F0C94641180918A02882319F081503E
:1024800080938A026091860270918702809188020F
:10249000909189020C94521180918A02833018F431
:1024A0008F5F80938A02609186027091870280918B
:1024B0008802909189020C9452119091860290FFAB
:1024C0003DC09170811129C092609093860266236D
:1024D00051F06091860270918702809188029091FC
:1024E00089020E94521160918602669570E04BE06D
:1024F00050E08CE091E00E94C828892BA9F010924E
:10250000250281E08093210220E0409189026091C0
:102510008802809187020C946411853210F09864CF
:10252000D4CF880F982BD1CF81E0809325020E94D1
:10253000EC0490931F0280931E02E3CF08958091D4
:1025400086028695815009F484E261E00C945D1264
:102550008091860286958F5F853208F081E061E088
:102560000C945D129091860290FF07C09695981783
:1025700020F0961710F40C94A81261E00C945D12F0
:10258000E6E8F2E083E0808311828FEF8283838329
:10259000148260817181828193810C945211109216
:1025A000F60180911A01E0E9F1E0882359F0809169
:1025B000970287FF07C08EE1DF011D928A95E9F738
:1025C0000C94C70A86E0F8CF1F93CF93DF93CDB763
:1025D000DEB7AA970FB6F894DEBF0FBECDBF83EC6F
:1025E00092E02091F100DC012D93CD01B2E08B3C13
:1025F0009B07B9F78091C402833009F472C0B8F424
:10260000813009F449C0823009F4B3C08091E800F8
:1026100083FF8BC28091C3029091C4029A3008F06C
:1026200084C2E92FF0E0EE50F74D0C9436288A3042
:1026300009F48EC08B3009F471C0893039F780916C
:10264000C302813219F78091C7029091C8020097A6
:1026500011F00297D9F68091E800877F8093E80017
:102660008091E80082FF38C09091F3008091F200E1
:10267000029731F48091F100813011F0863021F41D
:102680008091F10080939E028091E8008B77809387
:10269000E8000E94C903BACF8091C302813A09F0D1
:1026A000B5CF8091E800877F8093E8008091C702D2
:1026B0009091C802892B61F460E28FE992E070E0AA
:1026C0000E947B048091E8008B778093E8009ECF86
:1026D00060E090E080E0F3CF8091C1028111C0CF33
:1026E00095CF8091C302813A09F090CF8091C702C3
:1026F0009091C802892B09F089CF8091E800877FEB
:102700008093E8008091E80080FFFCCF80911A015F
:102710008093F1008091E8008E77B9CF8091C30259
:10272000813209F073CF8091C7029091C802892B42
:1027300009F06CCF8091E800877F8093E8000E94C9
:10274000C9038091C50280931A010E94CF125ECF07
:102750008091C302813209F059CF8091E800877FD0
:102760008093E8000E94C9038091C60280939D0275
:102770004DCF8091C302813A09F048CF8091E800A3
:10278000877F8093E8008091E80080FFFCCF8091F4
:102790009D02BECF803899F0823809F0C6C1809181
:1027A000C7028F70873008F0C0C18093E900809124
:1027B000EB0085FB882780F91092E90006C0809124
:1027C000BF029091C002911182609091E800977FC2
:1027D0009093E8008093F1001092F1008091E8005E
:1027E0008E779FC1882309F48DC1823009F09DC185
:1027F0008091C502811190C18091C7028F702FEF27
:10280000280F263008F091C18093E9002091EB0059
:1028100020FF82C1933031F48091EB00806280937D
:10282000EB007AC19091EB0090619093EB0021E076
:1028300030E001C0220F8A95EAF72093EA00109257
:10284000EA008091EB008860EACF81116EC110919F
:10285000C5021F778091E3008078812B8093E3008D
:102860008091E800877F8093E8000E94C9038091EF
:10287000E80080FFFCCF8091E30080688093E30054
:1028800082E0111183E08093C1024FC180588230F1
:1028900008F04BC12091C5023091C6022C3DE3E007
:1028A0003E07A1F583E08A838AE289834FB7F894D3
:1028B000DE01139620E03EE051E2E32FF0E050937A
:1028C0005700E49120FF03C0E295EF703F5FEF7087
:1028D0008E2F90E0EA30C0F0C7968D939D932F5FC6
:1028E000243159F74FBF8091E800877F8093E8003B
:1028F0006AE270E0CE0101960E947B048091E800BC
:102900008B778093E80011C1C096E7CF8091C70212
:102910009091C802432F55274330510509F44AC00E
:1029200078F54130510509F47AC08BE590E0EBE78A
:10293000F5E04230510509F0F8C02091E800277F0A
:102940002093E8002091C9023091CA0282179307B0
:1029500008F49C0140E02115310509F065C04111E2
:1029600063C08091E80082FDC9CF8091C1028823B5
:1029700029F2853019F28091E80083FFF2CFBECFB3
:102980004132510509F43CC04232510509F0CDC035
:102990008330910508F0C9C0FC01EE0FFF1FE1581C
:1029A000FE4F0190F081E02D84589E4FDC018C9108
:1029B00090E01AC0332721303105D1F021153105BF
:1029C00061F02230310509F0B0C0E8EEF5E0E491A5
:1029D0008E2F90E0E8EEF5E007C0E8E0F6E0E49145
:1029E0008E2F90E0E8E0F6E0009709F49EC0A5CFB6
:1029F000E8EFF5E0E4918E2F90E0E8EFF5E0F4CF1A
:102A00008330910508F091C0880F991FFC01EB57A6
:102A1000FE4F0190F081E02D89E090E08ECF82E1C1
:102A200090E0E6EDF5E089CF8091C102882309F4BA
:102A300065CF853009F462CF8091E80083FD5ECFD9
:102A40008091E80082FD8DCF8091E80080FF83CFE8
:102A50009091F3008091F2002115310519F0883032
:102A6000910550F041E0089709F040E08091E800BE
:102A70008E778093E8006FCF44914093F1003196B8
:102A8000215031090196E8CF803809F04EC080917D
:102A9000E800877F8093E8008091C2028093F10074
:102AA0009DCE811142C01091C5021230F0F5809187
:102AB000E800877F8093E8001093C2020E94C90358
:102AC000112311F084E005C08091E30087FDFACF67
:102AD00081E08093C10242E061EC81E00E94E80362
:102AE00042E261EC84E00E94E80342E261EC82E0B1
:102AF0000E94E80342E260EC83E00E94E8038091D8
:102B0000C10213C08091C502813079F481E0933015
:102B100009F080E08093C0021092E9008091E80003
:102B2000877F8093E8000E94C9038091E80083FFBB
:102B30000AC08091E800877F8093E8008091EB00D5
:102B400080628093EB00AA960FB6F894DEBF0FBEAA
:102B5000CDBFDF91CF911F91089569EE7EEF90E098
:102B600080E00E94B22860E082E090E00E94942819
:102B700060E083E090E00E9494281092F80160E009
:102B800084E090E00E94942860E082E290E00E945D
:102B9000942860E085E090E00E94942860E086E060
:102BA00090E00E9494286FEF87E090E00E949428C4
:102BB00040E050E0BA0188E090E00E94A62860E082
:102BC0008DE090E00E94942840E050E0BA0188E156
:102BD00090E00E94A62860E087E190E00E9494289F
:102BE00040E050E0BA018CE190E00E94A62870E03D
:102BF00060E080E290E00E94B22840E050E0BA013C
:102C000088E190E00E94A62880E00E944D100E947A
:102C1000651040E050E0BA018FE090E00E94A628E5
:102C200040E050E0BA0183E190E00C94A6283F9286
:102C30004F925F926F927F928F929F92AF92BF92CC
:102C4000CF92DF92EF92FF920F931F93CF93DF9378
:102C500000D000D00F92CDB7DEB78C01FC0183818C
:102C60009481892B31F08081918189238F3F09F0F4
:102C7000F6C50F900F900F900F900F90DF91CF91AE
:102C80001F910F91FF90EF90DF90CF90BF90AF908A
:102C90009F908F907F906F905F904F903F9008959E
:102CA0000E94C910F82E682F89819A810E94990A82
:102CB00069817A818F2D0E94BC107C01F80182818C
:102CC000882309F499C5C70182519F45409708F0B0
:102CD00051C58FEF93E00E948028FEEEEF0E57E182
:102CE000852E992493948823A1F18091F301877014
:102CF00009F4BFCFF8018281882309F4BACF80910B
:102D0000980282FDB6CF82E00F900F900F900F9047
:102D10000F90DF91CF911F910F91FF90EF90DF9077
:102D2000CF90BF90AF909F908F907F906F905F906B
:102D30004F903F900C94FF0A811424E09206A9F270
:102D4000C4010E948028811101C0EA943FEF831AD8
:102D5000930AE110F1CF1C821B82442443944AE081
:102D6000342E74018FEFE81AF80AC4010E948028FB
:102D700089831A82882309F4B8CF9FEF980F933084
:102D800000F58A83498292E0890E911CC7010E9456
:102D900080288B83882309F4A8CFFE0131967F0118
:102DA000F70120812223E9F2213009F049C0918105
:102DB0008281913041F4F2E0EF0EF11C0E94680F25
:102DC00009C04701EACF923049F422E0E20EF11C3B
:102DD0000E94B30E3FEFE31AF30AE2CF933031F4CF
:102DE00032E0E30EF11C0E943B0BF4CF943021F053
:102DF0008FEFE81AF80AEECF92E0E90EF11C30E00E
:102E000020E0B7016F5F7F4FF70141818053990B3D
:102E10008A30910550F021503109E0F28FE99FE0AE
:102E20000197F1F700C00000F6CF329EF001339E0B
:102E3000F00D11249C012E0F3F1F842F7B01E1CF49
:102E4000E22FF0E0EC50FE4F5490822F869586954D
:102E5000869590E0FC01EC51FE4F64902770712C38
:102E6000022E02C0759467940A94E2F7E1E06E22A4
:102E70007724FC01EC52FE4FA490B12C022E02C02C
:102E8000B594A7940A94E2F7F1E0AF22BB24FC01C9
:102E9000EC53FE4FC490D12C02C0D594C7942A9510
:102EA000E2F721E0C222DD246114710419F081EE01
:102EB0000E94B30EA114B10419F086EE0E94B30E65
:102EC000852D0E94680FAB2819F086EE0E943B0BFF
:102ED000672819F081EE0E943B0BCD2809F47ACFC8
:102EE0008CE26CCF81E00E941B0B03C081E00E944A
:102EF000F30A0E94E80AF9CE82E0F5CF82E0F7CF2C
:102F00002FEBE2162CE5F20609F44BC0A0F180ECA1
:102F1000E8168CE5F80609F04EC490918B02892FD3
:102F20008695869586958F5F8F719770843008F0AF
:102F300059C0880F880F880F892B80938B0280914E
:102F40008B0210C083E00E94D40580918B020E9406
:102F50007410CBCE80918B02982F987FE9F1885026
:102F600080938B02887F91E009F490E080918B023E
:102F700090FB80F913C080918B02982F96959695BF
:102F80009695933040F49F5F990F990F990F877032
:102F9000892B80938B0280918B02816080938B02BE
:102FA00019C080918B0280FF09C08E7F80938B02B5
:102FB0000E94741080E00E94300597CE80FD95CE6F
:102FC000816080938B02813019F489E080938B02B9
:102FD00080918B020E94741080918B028695869559
:102FE0008695E9CF90938B02AACF27E245EE65EE56
:102FF000FFC326E241EE60EEFBC327E245EE64EE3E
:10300000F7C326E241EE62EEF3C328E241E0EFCFE0
:10301000F1E6EF16FDE5FF0609F447C58091F601DC
:1030200096E1E9169CE5F90609F02AC48A7A91E04E
:1030300009F490E09093AE018111FEC089E20E94F4
:10304000320A0E94C20951CE86E0E8168CE5F806E5
:1030500009F4B7C080919702886097E0E9169CE573
:10306000F90608F49DC080919702806299C0809112
:1030700097028D7FECE0EE16ECE5FE0609F490C0B9
:1030800078F4809197028C602AE0E2162CE5F20633
:1030900009F486C008F49DC0809197028E7F80C09D
:1030A0008EE0E8168CE5F80609F499C08091970245
:1030B0008B7F9FE0E9169CE5F90608F471C08091CA
:1030C00097028F7E6DC0ECEFEE16ECE5FE0609F47C
:1030D0008AC0A0F524E1E2162CE5F20609F49BC0B3
:1030E00098F482E1E8168CE5F80609F484C0809132
:1030F00097028F7B93E1E9169CE5F90608F450C02E
:1031000080919702837F4CC0EAEFEE16ECE5FE0655
:1031100009F44DC008F051C025E1E2162CE5F20695
:1031200009F0F0C48091970282FB992790F921E081
:10313000922790FB82F990FB83F932C0E1143DE5C0
:10314000F30609F45EC0A0F48091980283609EEFBC
:10315000E9169CE5F90671F1809198028D7FEFEFF9
:10316000EE16ECE5FE0630F1809198028C7F22C0CD
:10317000F2E0EF16FDE5FF0609F45CC008F454C068
:1031800031E6E3163DE5F30609F0BCC490919702E1
:10319000892F8F7E94FF806103C0809197028160A8
:1031A00080939702AFC4809197028460F9CF809199
:1031B0009802816080939802A5C4809198028260F1
:1031C000F9CF809197028061EBCF80919702806464
:1031D000E7CF0E94CF12809197028068E1CF809163
:1031E0009702877FDDCF809198028E7FE3CF809119
:1031F00097028F7DD5CF0E94CF12809197028F7753
:10320000CFCF80919802982F909591708E7F892BC7
:1032100090FB81F9CFCF0E94CF1290919702892F16
:1032200097FB87F98058BCCF61E08EE090E00E9468
:10323000942868C460E0F9CF85E301CF85E30CC32F
:103240008091860280FF1BC08E7F809386026091F2
:1032500086027091870280918802909189020E9473
:10326000521110922502EFEFF0E722E0E150F0401A
:103270002040E1F700C000000E94480C36CD81607C
:103280008093860261E086950E945D122ECD4FE903
:1032900052E168EA72E10E94EA0527CD48EA52E16C
:1032A0006FE972E1F8CF42E352E169E272E1F3CFF4
:1032B00041E152E16DE172E1EECF49EF51E165E0AC
:1032C00072E1E9CF45E052E169EF71E1E4CF4CE40E
:1032D00052E16BE372E1DFCF61E081E0D5CF65E0E1
:1032E00082E00E94B21201CD68E086E0FACF64E18C
:1032F0008FE0F7CF67E185E1F4CF62E289E1F1CFBA
:1033000061E083E2C1CFFBE5EF16FDE5FF0611F1B9
:103310002CE5E2162DE5F20609F0E4C28091980250
:1033200082FB882780F991E089270E947910DAC210
:103330000E94CF123FEF84E39CE0315080409040E8
:10334000E1F700C000000E94240C0E94AD15CDCC16
:1033500081E0EBCF80E0E9CFC7010E94700AD82E50
:10336000D0C22F2D2F70C22E8F2D807F19F0C294C6
:1033700090EFC922DD20B9F0CC2069F080E28E0DFB
:10338000883010F0811009C08091F601C82AC092DF
:10339000F6010E94C2098E2D4DC08091F501C82A08
:1033A000C092F501F6CF8E2D0E943B0BCC2009F484
:1033B00043C080E28E0D883010F0811004C08C2D47
:1033C0000E94BB0906C0C0948091F501C822C0923A
:1033D000F5010E94C20930C03F2D3F70C32E8F2DD2
:1033E000807F803219F0C29480EFC822882089F053
:1033F00081E0881609F47FC0DD2009F489C0BB2074
:1034000009F47FC0F801858180FFC5CF8F70858367
:1034100078C02091980222FF4BC0DD2009F442C001
:10342000CC2039F08091F601C82AC092F6010E94A2
:10343000C20980E00E94B30E292D2850330B24309E
:10344000310510F40E942405AA2009F412CC8091C1
:10345000F30180FD0ECCF801128285958595859546
:103460000E941B0BC8010E9417168091F3018595DD
:10347000859585950F900F900F900F900F90DF918D
:10348000CF911F910F91FF90EF90DF90CF90BF9061
:10349000AF909F908F907F906F905F904F903F90F4
:1034A0000C94F30A80E00E943B0BCC2029F287CFDA
:1034B000DD20A1F09091F7018C2D892BB11003C074
:1034C0000E94310BB9CFE1E0BE12FACF22FDB4CF9A
:1034D000981709F4B1CF8093F701AECFB11006C0B1
:1034E0000E94B5098C2D0E942A0BA6CFF1E0BF16D1
:1034F00009F4A2CFF5CFDD2031F025E02B1508F43B
:103500009BCF8C2DDDCF34E03B1508F495CFEACF6F
:10351000BB2041F3F9E38F1209C02FEF37EE83E0B0
:10352000215030408040E1F700C000008E2D0E9405
:103530003B0B82CF8F2D86958695837061F081300D
:1035400009F07ACFC7019370D11002C090E080E0FB
:103550000E94F80471CFC7019370D11002C090E0AF
:1035600080E00E940E0568CF8E2DDD2029F00E949C
:1035700077070E94950660CF0E94BC06FACF8F2D78
:10358000837091F5D11058CF4E2D429546954770D6
:10359000440F440F8E2D8F70042E01C0880F0A94A3
:1035A000EAF72E2D2071E4FE07C02FE030E001C0C5
:1035B000220F4A95EAF720953F2D369536953370C0
:1035C000323069F050F44091F801313029F0822B0B
:1035D00084230E94260B30CF842B822BFACF282BFA
:1035E0008091F8018227F5CF8695DD2011F08F2D8F
:1035F0008170882309F420CF4E2D4295469547705F
:10360000440F440F8E2D8F70042E01C0880F0A9432
:10361000EAF72E2D2071E4FE07C02FE030E001C054
:10362000220F4A95EAF720953F2D3695369533704F
:10363000323069F050F44091CE02313029F0822BC3
:1036400084230E94E40AF8CE842B822BFACF282B05
:103650008091CE028227F5CF9F2D9F70F92EDD201D
:1036600029F0892F0E941B0B8E2D2ACF8E2D0E94B0
:103670002A0B8F2D0E94F30ADFCE8E2DE2EF8E16DD
:10368000B1F1E81570F0F0EF8F16D1F021EF82164E
:1036900091F0DD2009F45EC0B1107DCE8F2D8F71C9
:1036A0002AC033EF831651F194EF8912F2CF809143
:1036B000980282FF2FC08F2D8F71DD20D9F21BC0A1
:1036C000DD2081F0E4E0EB1508F4B6CE2F2D2F714C
:1036D00081E090E001C0880F2A95EAF79091CE0230
:1036E0008927AFCFF5E0FB1508F4A6CEEFCF8F2DDD
:1036F0008F71D110BFCF0E941B0B9ECE80E0DD20CA
:1037000009F49FCF9F2D9F7181E001C0880F9A958A
:10371000EAF797CFDD2099F02F2D2F71F22E822F0F
:103720000E941B0B8091980282FD07C038E0F39E37
:10373000C001112483608093F3018F2DDCCF81E0E1
:103740000E94FF0A81E08B1508F076CE82E00E948D
:10375000FF0A72CEBB2059F0893309F0E7CE9FEF04
:10376000E7EEF3E09150E040F040E1F7DDCE8F2D41
:103770008F7180CFF0E1EF16FFE5FF0609F4B2CBC1
:1037800021E1E2162FE5F20609F4B6CB8DEBE8163F
:103790008CE5F80609F4DECB08F0B2CBEBEBEE16C5
:1037A000ECE5FE0609F4CECB80E0FCEBEF16FCE581
:1037B000FF0609F4C8CB23EFE2162CE5F20609F464
:1037C00018CC08F051C188EDE8168CE5F80609F42C
:1037D0000CCC99EDE9169CE5F90609F416CCE7ED59
:1037E000EE16ECE5FE0609F04DC126E241EE61EE73
:1037F000C8010E94850F79CA30E1E3163FE5F30660
:1038000009F474CB81E1E8168FE5F80609F476CB6C
:1038100083EFE8168CE5F80609F4EBCB08F082C1DB
:10382000E8EDEE16ECE5FE0609F4DFCBF9EDEF1658
:10383000FCE5FF0609F4E9CB27EDE2162CE5F206DC
:10384000A1F2F6E1EF16FCE5FF0609F04BC080910E
:10385000AE018111F3CC89E20E94070AF2CB85E028
:10386000DE01119601900D928A95E1F7F80122810F
:1038700089819A81211114CA0E94700AF82E18CAEF
:1038800082722CECE2162CE5F20609F420CD08F049
:10389000ABC096ECE9169CE5F90609F404CD08F0F6
:1038A0007AC0F3ECEF16FCE5FF0609F4F0CC08F063
:1038B00061C032ECE3163CE5F30609F4C1CC3AE50D
:1038C000E3163DE5F30609F443CD08F01CCDE11401
:1038D0009CE5F90609F42CCDEEEDEE16ECE5FE06BE
:1038E00009F433CDF8018281E080F180882309F466
:1038F00033CDC7010E94C910D82E682FC7010E947E
:10390000990AB7018D2D0E94BC100E942D087C01E0
:10391000882EF801D280B580B2943FE0B322809126
:10392000F3018770C1F0AD2CDD20B1F08F2D807FC9
:10393000803421F080E28E0D883068F0809198020A
:1039400082FD09C082E00E94FF0A8091F301877026
:10395000AA24A3948111A12C9F2C92942FE092224F
:10396000FBE0F91508F468CDE92DF0E0E450F74DDF
:103970000C94362894ECE9169CE5F90609F48ECCF3
:1039800049E252E162E372E1E5ECEE16ECE5FE0697
:1039900009F481CC94CFF9ECEF16FCE5FF0609F4AD
:1039A0008CCC88F437ECE3163CE5F30609F480CCC4
:1039B0004DE152E161E172E198ECE9169CE5F9060E
:1039C00009F469CC7CCFEAECEE16ECE5FE0609F4CE
:1039D00079CC4BE352E16CE472E1FBECEF16FCE5D1
:1039E000FF0609F458CC6BCF21EDE2162CE5F20668
:1039F00009F47DCCB8F48EECE8168CE5F80609F4F1
:103A00006ECC08F469CCEFECEE16ECE5FE0609F49A
:103A10006BCC6EE089E0F0EDEF16FCE5FF0609F4F3
:103A200060CC4DCF24EDE2162CE5F20609F465CC0E
:103A300078F482EDE8168CE5F80609F45BCC61E0D9
:103A400088E193EDE9169CE5F90609F41DCC37CF22
:103A5000E5EDEE16ECE5FE0609F452CCFDE5EF16B9
:103A6000FF0609F442C92BCFF5EFEF16FCE5FF0680
:103A700009F4C7CA08F4C1CA36EFE3163CE5F306F9
:103A800009F45EC01092CD0293E0E9169DE5F906B7
:103A900008F0BECAEAEFEE16ECE5FE0630F4C70108
:103AA00082509C45449708F0B9CA0E9444119093F3
:103AB00098028093970220E1E2162CE5F20609F4C1
:103AC00096CB08F000CB88E0E8168CE5F80609F400
:103AD0007CCB08F0CCCAE4E0EE16ECE5FE0609F477
:103AE00062CB08F0B1CA22E0E2162CE5F20609F436
:103AF00054CB80919702826033E0E3163CE5F306F5
:103B000009F44ECB60919702F090980284E090E027
:103B10000E9494286F2D82E290E00E9494280E94D7
:103B2000CF12E3C835EFE3163CE5F30609F469CAA2
:103B300008F463CA96EFE9169CE5F90609F081CE10
:103B400027E245EE66EE54CE1F93CF93DF9380912C
:103B5000C001807FA9F48091BD01882389F0809104
:103B6000F201D091C1016091BB017091BC01A091A3
:103B7000BE01B091BF01C62FC72316E0D81304C001
:103B8000DF91CF911F91089590E0109711F0CF3FF2
:103B900019F401968770F2CF189F9001199F300D8C
:103BA0001124F901EE53FE4F41814713F2CF4081BA
:103BB0004613EFCF42814111ECCF438154814A1B20
:103BC0005B0B483C510528F78091C0018F708061E4
:103BD0008093C001F901E953FE4F80818F708061AD
:103BE00080838BEB91E00E941716DF91CF911F919C
:103BF0000C94660AAF92BF92CF92DF92EF92FF923F
:103C00000F931F93CF93DF93CDB7DEB761970FB6B6
:103C1000F894DEBF0FBECDBF8C0185E0F801DE0158
:103C20001D9601900D928A95E1F7F801E2808BEBE9
:103C3000A82E81E0B82E6091BE017091BF01611580
:103C4000710509F432C19091BB014091BC01892FEB
:103C500084238F3F09F429C120813181C380D4801E
:103C6000F090BD01F601E61BF70BFF2009F4E8C058
:103C70008091C001582F507FE83CF10508F0ABC09F
:103C8000511177C0FE2C431321C092131FC0E110C5
:103C90001DC08F7080618093C001C5010E941716FE
:103CA0008091C001F80185838F2D61960FB6F8943D
:103CB000DEBF0FBECDBFDF91CF911F910F91FF905F
:103CC000EF90DF90CF90BF90AF900895CD2829F06E
:103CD000822F83238F3F09F003C180E0F82FF1701A
:103CE000DF2E80FF3CC08091F2014091C10156E07F
:103CF000841315C02D873E878D859E850E94F81000
:103D0000292F22952F702230F0F0243018F59F7063
:103D1000F1F0F8019581907FD1F4D12C1EC090E094
:103D2000589FF001599FF00D1124EE53FE4F618111
:103D3000361306C06081261303C06281E6120FC0ED
:103D400001968770D5CF9F7011F0882331F3805E84
:103D5000883018F3C8010E941716FD2CA5CFEE205D
:103D600009F4A2CF8091C00181608093C001F12C41
:103D70009BCF431306C0921304C0F801EE2009F450
:103D800079C0C8010E940411882309F1EE20F9F0DE
:103D90008091C001803270F02091BB013091BC0154
:103DA00038872F831986DB86CA868C87CE010796D3
:103DB0000E94171686E0F801ABEBB1E001900D927E
:103DC0008A95E1F70E94A41DFF24F3946DCFC801EA
:103DD0000E941716F9CF51110AC08BEB91E00E9497
:103DE000171686E0F50111928A95E9F7C0CF4313C3
:103DF0000FC092130DC0E1100BC0F8018583C801FC
:103E00000E94171686E0F50111928A95E9F74CCFCA
:103E1000C8010E9404118823D1F2EE20C1F28091E2
:103E2000C001803238F22091BB013091BC013A834D
:103E300029831B82DD82CC828E83CE010196B8CF8E
:103E4000E83CF105F8F6FE2CEE2009F243131FC002
:103E500092131DC08091C00180FD10C0982F907FEB
:103E600069F0F8018583903F31F0982F907F905F43
:103E70008F70892B8583C8010E94171686E0F80190
:103E8000ABEBB1E001900D928A95E1F70DCFC8013F
:103E90000E94041181118ECF8091C00181608093B6
:103EA000C001C8010E941716FFCEEE2009F48FCF83
:103EB000C8010E940411F82E882309F488CF86E0F7
:103EC000F801ABEBB1E001900D928A95E1F780919A
:103ED000BB019091BC010E94F8100E94A41DE4CE89
:103EE00081E08E25FBCE1F93CF93DF93CDB7DEB756
:103EF00067970FB6F894DEBF0FBECDBF4B8B5C8BC0
:103F00006D8B7E8B8F8B61111092F5011A8A198A45
:103F100085E0FE017396DE011D9601900D928A9553
:103F2000E1F786E0FE013D96DE01179601900D92C5
:103F30008A95E1F7CE0107960E94FA1D882389F041
:103F400016E08091F2019091C101891349C06796F2
:103F50000FB6F894DEBF0FBECDBFDF91CF911F919A
:103F6000089586E0FE013796DE01119601900D92CC
:103F70008A95E1F78A859B85892B11F38F81988536
:103F800089238F3FE9F22091C10130E0C9010196F8
:103F9000877099274091F2014817190671F40E9421
:103FA000CF121092C1011092F20186E0EBEBF1E02A
:103FB000DF011D928A95E9F7C3CF96E0929FD00169
:103FC000939FB00D1124AE53BE4FFE013196019068
:103FD0000D929A95E1F78093C1010E94660AB0CFD5
:103FE000819FC00111248E539E4F0E94FA1D882389
:103FF00009F4ADCF8091F20190E001968770992786
:104000008093F2019ECF7F928F929F92AF92BF9248
:10401000CF92DF92EF92FF920F931F93CF93DF9394
:1040200000D000D000D0CDB7DEB78E010F5F1F4F9C
:1040300086E0D8011D928A95E9F78CE4882E81E00C
:10404000982E91E5E92E91E0F92E77247394CC24F3
:10405000C394D12C37E5A32E31E0B32EF401819126
:104060004F018F3F09F443C0F894E82FE295EF70B9
:10407000F0E021A18F70A60102C0440F551F8A9560
:10408000E2F7CA01922F982B91A392A180958923E0
:1040900082A3789400C061E571E0F801472D409556
:1040A000DB019D91BD0180819F3F09F467C0292FED
:1040B00022952F7030E0D90190962C9130E09F70BE
:1040C00002C0359527959A95E2F720FD57C08729BC
:1040D00080833196A616B70619F7F40131978081CF
:1040E0008F3F11F00E94D307B0EABA95F1F7770C31
:1040F000E814F90409F0B2CF46E050E0B8018CEFC3
:1041000091E00E94D528FF24F394009709F4F12C44
:10411000892BB1F186E0F801ACEFB1E001900D928E
:104120008A95E1F781E08093FB010E94EC04909373
:10413000FA018093F9018091F9019091FA010E94AE
:10414000DD04059708F18091FC0180930B028091BA
:10415000FD0180930C028091FE0180930D028091FD
:10416000FF0180930E028091000280930F028091E4
:104170000102809310021092FB0106C08423A8CF95
:104180008091FB018111D7CF8F2D26960FB6F89421
:10419000DEBF0FBECDBFDF91CF911F910F91FF907A
:1041A000EF90DF90CF90BF90AF909F908F907F90D7
:1041B000089590E080E00E948E28893E9E4F11F481
:1041C0000C942B1180E008950E94D92081110AC01F
:1041D0000E94AD1580918B028470896180938B025F
:1041E0000E94741086E090E00E94802880938B02E9
:1041F000803220F08770886180938B0290918B02CF
:10420000892F817090FF04C0892F869586958695A9
:104210000C9430051F920F920FB60F9211242F931A
:104220003F934F935F936F937F938F939F93AF933E
:10423000BF93CF93DF93EF93FF93D091E900DF70AB
:104240008091EC00C82FC17080FDC0E81092E90099
:104250008091F000877F8093F00078940E94E412B0
:104260001092E9008091F00088608093F000CD2BDF
:10427000CF70C093E900FF91EF91DF91CF91BF9193
:10428000AF919F918F917F916F915F914F913F91EE
:104290002F910F900FBE0F901F9018951F920F92A5
:1042A0000FB60F9211242F933F934F935F936F9309
:1042B0007F938F939F93AF93BF93EF93FF938091DF
:1042C000E10082FF09C08091E20082FF05C0809179
:1042D000E1008B7F8093E1008091DA0080FF24C0B1
:1042E0008091D80080FF20C08091DA008E7F80937B
:1042F000DA008091D90080FF9DC080E189BD82E114
:1043000089BD09B400FEFDCF81E08093C102809198
:104310009C02811109C00E944F030E941A048091DF
:10432000E20084608093E2008091E10080FF17C08A
:104330008091E20080FF13C08091E2008E7F809325
:10434000E2008091E20080618093E2008091D800D9
:1043500080628093D80019BC85E08093C10280916F
:10436000E10084FF2BC08091E20084FF27C080E140
:1043700089BD82E189BD89B5982F917080FFFBCFFF
:104380008091D8008F7D8093D8008091E1008F7E4E
:104390008093E1008091E2008F7E8093E200809123
:1043A000E20081608093E2008091C202882309F4D8
:1043B00047C084E08093C1028091C1028091E100F6
:1043C00083FF27C08091E20083FF23C08091E1003A
:1043D000877F8093E10082E08093C1021092C20245
:1043E0008091E1008E7F8093E1008091E2008E7FDA
:1043F0008093E2008091E20080618093E20042E0DD
:1044000060E080E00E94E8038091F0008860809383
:10441000F000FF91EF91BF91AF919F918F917F91AC
:104420006F915F914F913F912F910F900FBE0F9021
:104430001F90189519BC1092C10210929C0274CF63
:104440008091E30087FD93E09093C102B5CF78940B
:104450001F921FB61F9211248F939F93AF93BF9308
:104460008091930290919402A0919502B09196024E
:104470000196A11DB11D8093930290939402A09385
:104480009502B0939602BF91AF919F918F911F902B
:104490001FBE1F9018951F921FB61F9211248F9355
:1044A0009F93AF93BF9380919202811113C080912B
:1044B000930290919402A0919502B0919602419638
:1044C000A11DB11D8093930290939402A093950235
:1044D000B0939602BF91AF919F918F911F901FBE95
:1044E0001F901895CDB7DEB7AA970FB6F894DEBF28
:1044F0000FBECDBF84B7877F84BF0FB6F894A89551
:1045000080916000886180936000109260000FBE0F
:1045100080E890E00FB6F89480936100909361007A
:104520000FBE85B7806885BF85B7806885BF81ED80
:1045300097E090938D0180938C010E944F030E941D
:104540001A048091E20084608093E2007894809164
:10455000C1028823A1F01091E9001F709091EC0036
:10456000892F817090FD80E8182B1092E9008091CE
:10457000E80083FD0E94E4121F701093E90082E0BE
:1045800084BD93E095BD9AEF97BD80936E000E9425
:104590002B11811102C00E9465100CE411E031E57D
:1045A000E32E31E0F32ED8018D918D018F3F11F074
:1045B0000E94D307E016F106B1F701E511E027E507
:1045C000E22E21E0F22EF80181918F018F3F11F050
:1045D0000E94D307E016F106B1F786E0EBE0F2E0C7
:1045E000DF01282F1D922A95E9F7ECEFF1E0DF01BA
:1045F0001D928A95E9F70E94D920811102C00E947C
:10460000AD1582E090E00E948028809304020E9411
:10461000441190939802809397020E940320EFE345
:10462000FCE93197F1F700C000000E94032080915F
:104630000B0280FF08C06FEF7FEF90E080E00E94E8
:10464000B2280E94240C83E090E00E9480280E94FF
:10465000260B269A2E9882E28093800089E180932F
:1046600081008FEF9FEF90938700809386000E94D8
:10467000E4200E94E42080910202811133C00E9454
:10468000D920811104C00E94AD150E94C01288E09B
:1046900090E00E948828609386027093870280933E
:1046A0008802909389026E7F71F40E94C01288E0A4
:1046B00090E00E948828609386027093870280931E
:1046C0008802909389020E94F00510922502809141
:1046D000860280FF04C060E086950E945D1281E042
:1046E0008093020280E091E090938F0280938E028B
:1046F00008E1E02EF12C8BE092E096E0D92ED80E66
:104700008091C10210E4B12E00E112E1853009F47C
:10471000ABC10E940320882359F08FB7F8944091D1
:1047200093025091940260919502709196028FBF0E
:10473000ABE0B2E0E5E0F2E010E000E0302F8D9178
:104740009191981709F4A1C1292F282790E0BB2443
:10475000B3944B2D422309F493C199A33AA38B211F
:1047600091E009F490E09BA30E94EC048160782F13
:104770009DA38CA349A15AA16BA18DA10E94731F77
:10478000F801EB5FFD4F8081B826B0828091250251
:104790008823D1F180912402E0918602E695E81BFE
:1047A000E0932002823009F087C1F0E0EE57FD4F20
:1047B000E4910E2F10E0BFE9AB2EBEE0BB2E80913E
:1047C0002102882361F0109221020E94EC04909350
:1047D0001F0280931E0210922302109222020E9456
:1047E000EC04E0911E02F0911F028E1B9F0B8F3F85
:1047F0009F4750F4E00FF11FF0931F02E0931E0259
:104800008EE192E0F501099586E0E8E1F2E0DE0153
:10481000119601900D928A95E1F7B0901A02A0903E
:104820001B0210911C0200911D0210921A0210929C
:104830001B0210921C0210921D028B2D8A2909F472
:1048400048C080911602909117020E94DD049C01DD
:1048500090911202992309F49CC323333105C8F1C6
:104860009F3F19F09F5F90931202BB2059F00E9466
:1048700057079FEF1B140CF491E0899F802D1124A2
:1048800080931A02AA2059F00E9457079FEF1A142A
:104890000CF491E0899F802D112480931B023091AC
:1048A0001A023323B1F020911B02222391F045EB31
:1048B0003403C0011124992309F458C190931A02BA
:1048C00045EB240390011124332309F453C13093A1
:1048D0001B02812F802B09F448C080911402909113
:1048E00015020E94DD049C0190911102992309F4A4
:1048F0004BC325363105C8F19F3F19F09F5F909358
:104900001102112359F00E9435079FEF11160CF484
:1049100091E0899F802D112480931C02002359F07F
:104920000E9435079FEF10160CF491E0899F802DAF
:10493000112480931D0230911C023323B1F0209189
:104940001D02222391F045EB3403C0011124992369
:1049500009F414C190931C0245EB24039001112427
:10496000332309F40FC130931D0280911A029091F4
:104970001B02892B90911C02892B90911D02892B7F
:1049800011F00E94950686E0FE013196A8E1B2E0A2
:1049900001900D928A95E1F70E94240590910302FF
:1049A000891721F00E942405809303028091C1029F
:1049B000843009F0A5CE83E08093E9008091E8007F
:1049C00082FF9ECE8091E80090E085FF06C00E94A5
:1049D0006E03882309F4DAC091E08091E8008B77B8
:1049E0008093E800992309F48BCEE981E150E3310B
:1049F00008F04EC1F0E0E85FF64D0C943628809147
:104A0000C102843021F180E00E94300510929202B0
:104A10000FB6F894A895E09260000FBEB0926000C7
:104A200083B7817F846083BF83B7816083BF7894BD
:104A3000889583B78E7F83BF0FB6F894A895809131
:104A40006000886180936000109260000FBE8091CA
:104A5000C002882349F00E940320EBE0F2E081913C
:104A6000811173C2DE12FBCF8091C102853009F43F
:104A7000C6CF0E94CF120E94E4200E94240549CE96
:104A80009F5FBB0C953009F064CE0F5F1F4F06305F
:104A9000110509F053CE8FEF8EA38FA318A60E94A5
:104AA000EC048160782F9AA789A74EA15FA168A521
:104AB0008AA50E94731F6ACE863059F4F0E0E1584F
:104AC000FD4FE4910E2F10E0AFE8AA2EAEE0BA2E13
:104AD00076CE893061F4E695F0E0E458FD4FE4913C
:104AE0000E2F10E0FBEFAF2EFDE0BF2E68CE8F3013
:104AF00061F4E695F0E0E758FD4FE4910E2F10E0E9
:104B0000EDE8AE2EEDE0BE2E5ACE853159F4F0E040
:104B1000EA58FD4FE4910E2F10E07FE3A72E7DE0D1
:104B2000B72E4DCE08E210E046EBA42E4CE0B42E9A
:104B3000883109F444CE833249F4E4E7F2E0059188
:104B4000149166E3A62E6EE0B62E39CE04EF11E086
:104B50005DE7A52E5CE0B52E843209F430CE00ED81
:104B600017E03FEEA32E35E0B32E29CE81E08093EF
:104B70001A02A6CE81E080931B02ABCE81E0809327
:104B80001C02EACE81E080931D02EFCE00E210E02D
:104B9000CE0101965C018091E80085FD0AC08091FC
:104BA000E8008B778093E8000E946E03882399F3D6
:104BB00013CF8091F100D5018D935D010150110952
:104BC00051F70ACF1A8289E08B832DC08A81823007
:104BD00009F4D1C18330A9F0813009F059C02FB751
:104BE000F894609193027091940280919502909153
:104BF00096022FBF0E943C286B837C838D839E830B
:104C000012C080910B028B8380910C028C83809167
:104C10000D028D8380910E028E8380910F028F830F
:104C20008091100288878091C102843009F068CD9C
:104C30001091E9001F709091EC00892F817090FD18
:104C400080E8182B82E08093E9008091E80080FFE3
:104C50000DC050E040E060E270E0CE0101960E949D
:104C60009F038091E8008E778093E8001F70109377
:104C7000E90046CD8A81823059F46B817C818D8137
:104C80009E810E943C2886E290E00E949428CBCF2F
:104C90008FEF8983C8CF4C816B818A810E949610E7
:104CA0009827892798279E838D83BDCFAD80BE80AE
:104CB000BA24AB24BA248A810B81BAE00B9F80010D
:104CC0001124ECE38E9F000D111D11248C8190E0C6
:104CD000880F991F080F191F6B2DC80187960E9416
:104CE00094286A2DC8018896D0CF0E94F90F9BCFD7
:104CF0008A81893061F48B81F3E08F9FC001112498
:104D00006FEF70E00E94EC27862F0E94D4058A8105
:104D10008138C1F060F4803809F085CF20E04B8104
:104D200060918802809187020E9464117CCF823852
:104D300059F1833809F077CF20E0409189026C81E6
:104D40008B81F2CF60E08B810E945D129B8180910C
:104D50008602911111C08E7F8093860210922502E7
:104D60002FEF40E782E0215040408040E1F700C053
:104D700000000E94480C57CF81608093860260E05B
:104D800086950E945D124FCF8B8180938A024BCF14
:104D90008A81893059F08A30C1F0813821F1B8F424
:104DA000803809F040CF809189020ECF80918B022C
:104DB000869586958695AFEF8A9FC001112463E0A2
:104DC00070E00E94EC276B832ECF1B822CCF8238A1
:104DD00091F0833809F027CF809187028B838091EF
:104DE00088028C8320CF8091860280FF02C0869546
:104DF000EBCE80E0E9CE80918A02E6CE80918B02F4
:104E00000E947410609186027091870280918802DE
:104E1000909189020E94521106CF80E18A8303CFCC
:104E200082E08A8389EED0CE0A811B811027012778
:104E30001027FE0131965F018C80CF01880D911DF6
:104E40004C01C801895E9E4F8A149B0409F4EBCE85
:104E5000093EA2E01A0750F40E948028F5018483DD
:104E60000F5F1F4FBFEFAB1ABB0AEBCFD5011496F4
:104E70001C92F6CF0A811B81102701271027FE0103
:104E800031964F01AC80A00EB12EB11CC801895ED5
:104E90009E4FA016B10609F4C6CE093EF2E01F07E8
:104EA00028F4D40114966C910E949428BFEF8B1AB9
:104EB0009B0A0F5F1F4FEACF0E94E90FB4CE84E038
:104EC000ADCF0A811B81102701271027FE013196E3
:104ED0005F018C80CF01880D911D4C01C801879620
:104EE000A814B90409F49FCE003F110558F40E949C
:104EF0008028D50114968C930F5F1F4FFFEFAF1AD8
:104F0000BF0AECCFF5011482F7CF0A811B8110276D
:104F100001271027CE0101964C01AC80A00EB12EC6
:104F2000B11CC8018796A016B10609F47CCE003FDB
:104F3000110528F4D40114966C910E949428BFEFB7
:104F40008B1A9B0A0F5F1F4FECCF09BD19BD09B427
:104F500000FEFDCF8091D8008F7D8093D800809196
:104F6000E00082608093E0008091E00081FDFCCF52
:104F70000E94CF1279CD86E290E00E9480281B82A9
:104F80001C821D828E834FCE2D32314008F0B6CC6C
:104F9000ECCC2D32314008F065CC9BCCDB018F93FB
:104FA0009F930E946128BF91AF91A29F800D911D98
:104FB000A39F900DB29F900D1124089587FB082E9A
:104FC000062687FD819567FD61950E9474280EF481
:104FD000919507FC81950895AA1BBB1B51E107C061
:104FE000AA1FBB1FA617B70710F0A61BB70B881F79
:104FF000991F5A95A9F780959095BC01CD01089508
:1050000097FB072E16F4009407D077FD09D00E9475
:10501000EC2707FC05D03EF4909581959F4F0895AD
:10502000709561957F4F0895A1E21A2EAA1BBB1BB4
:10503000FD010DC0AA1FBB1FEE1FFF1FA217B30764
:10504000E407F50720F0A21BB30BE40BF50B661F7A
:10505000771F881F991F1A9469F76095709580953E
:1050600090959B01AC01BD01CF010895EE0FFF1F8C
:105070000590F491E02D09946927962769277827F0
:105080008727782708950E944B28332312F48A1B20
:105090009B0B0C945C28A29FB001B39FC001A39FFF
:1050A000700D811D1124911DB29F700D811D112461
:1050B000911D08950E944B28B7FF0895821B930B02
:1050C00008950E944B28A59F900DB49F900DA49F1A
:1050D000800D911D11240895B7FF0C9461280E9442
:1050E0006128821B930B0895991B79E004C0991FD6
:1050F000961708F0961B881F7A95C9F78095089532
:10510000F999FECF92BD81BDF89A992780B508958F
:10511000A6E1B0E044E050E00C94BA28A8E1B0E089
:1051200042E050E00C94BA28262FF999FECF92BDA8
:1051300081BDF89A019700B4021639F01FBA20BD5C
:105140000FB6F894FA9AF99A0FBE08950396272F8E
:105150000E9495280E949428252F0E949528242F8C
:105160000C9495280196272F0E9495280C9494283A
:10517000DC01CB01FC01F999FECF06C0F2BDE1BD17
:10518000F89A319600B40D9241505040B8F7089506
:10519000FC014150504030F001900616D1F7319794
:1051A000CF010895882799270895FB01DC0104C0E9
:1051B0008D910190801921F441505040C8F7881B0F
:1051C000990B0895F894FFCF161116111F111F1196
:1051D00021111F111F111F111611161126111F1158
:1051E0001F112611CA13F2139515F21395152514E4
:1051F0004614951544155115B119B119EC19EC194E
:105200009A1AB41A1C1A1C1ABF1A2C1B3D1B3D1BE0
:10521000E225E6253A264B26562675267826C82608
:10522000FE26482648260D27102714273A275C27F4
:065230005F2761278527BE
:10523600DA04E40BC30BBF0BBB0BD90401191A1B11
:105246001C1D1E1F20212201020101818283E20012
:10525600E900EA00B500B600B700CD008301CC0036
:105266008A019201940121022302240225022602C8
:1052760027022A02B300B4006F0070009593929142
:1052860090949697343566000102020202060606DD
:105296000909090909090F0F0F0F0F0F1515151821
:1052A6001919191919191919191923244022B6841B
:0C52B600016201AC008D05A605C60500D4
:00000001FF
